:020000040000FA
:020000001128C5
:08000800A100030EA0000B088B
:100010000B1C0B2805088B01200E8300A10E210E5E
:100020000900831285010730990000308C000430EC
:10003000900083169F01850183128316FF23900091
:100040006400073081003A3085003A309500323044
:10005000960000308C0083128030D100B820050853
:100060008B018B158B1763008B018030D100B8207A
:100070000430D600851C49280530D200C220051561
:1000800005148030D100B8208518412805110510CD
:100090002C28F030D500D401D701851D2C28051E51
:1000A0006228851A2C281830D800852000380319BA
:1000B0002C280230D200C2205608D5000514852015
:1000C00005102C28851E2C28051A2C282830D8002D
:1000D0008520003803192C280230D200C22056088F
:1000E000D5000515852005112C286D22F4347939A9
:1000F0005010EB3A6F34273BA0397238E234ED30C0
:100100006131A039E13B653900171530D100B820C5
:100110000508F839D1000038031D9B28D708031DB6
:10012000D40A083054020319D403D70154085502E5
:10013000031D8528003451085806031DA2280130EC
:10014000D7008528D408031D00340134F020693914
:100150002036391932103018801AD00BAD2808001B
:100160006438E936723AC03CE136EC347217803AB2
:10017000D001D00BB928D10BB9280800B51A371A0D
:10018000311BB31AD001D101D00BC428D10BC42824
:06019000D20BC428080098
:0207FE00803445
:02400E00943FDD
:00000001FF
